:030000000235E5E1
:0C35E50078FFE4F6D8FD75817D02362CDD
:100EE20020000A3C2E2E2E3E004950436F6E6E6546
:100EF20063745245510A004950436F6E6E656374C4
:100F0200000A49504E6F41434B210A003E432C5682
:100F12002C43432CC0E4E0EFF2E5F020D1E8EDEA07
:100F2200EEEC49500A003E432C4D41432C25303211
:100F320062583A25303262583A25303262583A25A0
:100F4200303262583A25303262583A25303262588D
:100F52002C4D414320E0E4F0E5F10A003E432C56DB
:100F620045522C20332E3220EEF220257320257399
:100F72002CC2E5F0F1E8FF20495020ECEEE4F3EB5F
:100F8200FF0A004A616E203237203230313100319F
:100F9200363A34323A3430003E432C4C442C5052D0
:100FA2004F473A20202020202020202020202020CF
:100FB200202020202020202020202020202020202F
:100FC200202020202020202020202020202020201F
:100FD200202020202020202020202020202020200F
:100FE20020202020202020202CC4E0F2E020EFF05E
:100FF200EEF8E8E2EAE828F4E0E9EB290A003E2A02
:101002002C312CCEF1EDEEE2EDFBE520EFE0F0E04D
:10101200ECE5F2F0FB20F1E5F2E5E2EEE3EE20E8AA
:10102200EDF2E5F0F4E5E9F1E00A003E412C413051
:10103200312C2562752E2562752E2562752E25624C
:10104200752C495020E0E4F0E5F120E0E4E0EFF215
:10105200E5F0E00A003E412C4130322C2562752E2B
:101062002562752E2562752E2562752C495020E069
:10107200E4F0E5F120EEF1ED2E20F1E5F0E2E5F00D
:10108200E00A003E412C4130332C2562752E256248
:10109200752E2562752E2562752C495020E0E4F0EC
:1010A200E5F120F0E5E72E20F1E5F0E2E5F0E00AD7
:1010B200003E412C4130342C2562752E2562752E5E
:1010C2002562752E2562752CCCE0F1EAE020F1E56F
:1010D200F2E80A003E412C4130352C2562752E255E
:1010E20062752E2562752E2562752CD8EBFEE70AF5
:1010F200003E2A2C312CC4EEEF2E20EFE0F0E0EC83
:10110200E5F2F0FB20F1E5F2E5E2EEE3EE20E8EDB8
:10111200F2E5F0F4E5E9F1E00A003E422C53303109
:101122002C2562752CC6E4E0F2FC20E7E0EFF0EE3D
:10113200F1E020F1EEE5E4E8EDE5EDE8FF20EEF286
:1011420020F1E5F0E2E5F0E00A003E422C533032B5
:101152002C2562752CCEE1ECE5ED20F120F1E5F0D5
:10116200E2E5F0EEEC20E1E5E720EAE2E8F2E0ED8C
:10117200F6E8E90A003E422C5330332C2562752CE6
:10118200CFE5F0E5E7E0EFF3F1EA20EFF0E820EF5A
:10119200EEF2E5F0E520F1E2FFE7E820F120F1E5EB
:1011A200F0E2E5F0EEEC0A003E454E440A000A4445
:1011B200756D7058202020202030302030312030B2
:1011C2003220303320303420303520303620303752
:1011D2002030382030392030412030422030432026
:1011E2003044203045203046000A3A003A20000AB6
:1011F200000A44756D7044202020202030302030B9
:101202003120303220303320303420303520303617
:1012120020303720303820303920304120304220F1
:101222003043203044203045203046004572722041
:101232006B657900526420656570726F6D0A0052A9
:1012420064204D454D0A00526420436F64650A00D4
:10125200577269746520436F64650A00446562755C
:10126200674950204F4E0A00446562756749502015
:101272004F46460A00446562756755736572204F92
:101282006E0A00446562756755736572204F464663
:101292000A0044656275674D7367204F6E0A004409
:1012A200656275674D7367204F46460A00436F6E4D
:1012B200666967206C6F636B210A0057722065654F
:1012C20070726F6D0A0020536176652065657072D9
:1012D2006F6D210A00457272204D414321004C6F0F
:1012E20061643E3E002A003C4130313D003C4130C9
:1012F200323D003C4130333D003C4130343D003C06
:101302004130353D003C21003C5330313D003C53DF
:1013120030323D003C5330333D003C5330353D00CC
:061322003C5330363D0093
:063F100001130001110085
:103F4600C28E438910E4F58B758DB8D2ABD28E2222
:03001B0002355556
:10355500C0E0C083C082C0D0C28E758B00758DB8A7
:1035650020170675A61E75A6E10511D213E5136091
:10357500020513E512D39401400215120516E5164E
:10358500540F7048D21FE516543F7012D211906641
:103595008BE0600A04F0E0D394B44002D217906641
:1035A50086E0600204F0906104E0600214F0906629
:1035B5008CE0D394014003E014F03016020514E5C5
:1035C50015D394644004D21780020515E510D394F1
:1035D5000140021510D28ED0D0D082D083D0E032F7
:10087900C291C290D2B5C21C7D027C007F07123E94
:10088900F38F4DE54D646060097D017F60123E8EF6
:10089900D21CE4FDFC7F0B123EF38F4DE54D30E693
:1008A900097D04E4FF123EB2D21C7D017C007F0762
:1008B900123EF38F4DE54D7008FD7FFF123E8ED23B
:1008C9001C301C03126000C288C2A8C2AA75890024
:1008D90012390D90633EE0B4FA06A3E064CE607B62
:1008E900E4F54D7436254DF582E43463F583E4F07F
:1008F900054DE54DB443EC90633E74FAF0A374CE14
:10090900F0A374CCF0906344740AF0E4A3F0A30458
:10091900F0A3F090633A74FFF0A3F0A3F0E4A3F01E
:10092900906355740AF0E4F54DE54D2401FFE43375
:10093900FE7436254DF582E43463F583E0FD123EFD
:100949006A054DE54DC3944340DFE4F5A775A61E3E
:1009590075A6E1907FF0F0A3F080FE9063497403DF
:10096900F0A374CCF0E4906348F0123331C2B512AD
:100979003A73C217123C58D21CC21EC21D9065762A
:100989007408F09062B47424F0E4A3F090633EE03C
:100999009062B6F090633FE09062B7F0906340E0F8
:1009A9009062B8F0906341E09062B9F0906342E0E0
:1009B9009062BAF0906343E09062BBF0751201E473
:1009C900906577F0C218C219C21AC21B201C18AF51
:1009D9004DFE7D0312309CE4FF1233FB7E0E7FE255
:1009E900E4FBFDFC122CB390668BE060037401F00C
:1009F900E4906104F0F514906575F0F515123F4621
:100A090075A70775A61E75A6E1D2AFE4F515906125
:100A190004E0700312168490668CE06401701D90E6
:100A290080007410F09080A874FFF0A3F0A3F0A3E5
:100A3900F0E490668CF0D21CC21DC21E908008E0C2
:100A4900F54D30E405D2187410F0E54D30E508D2C3
:100A59001A9080087420F0E54D30E608D21990808C
:100A6900087440F0E514C394034019908002E4F03F
:100A7900908001F0908000F0E51494064006E4F5BA
:100A890014123C589080A0E07003123A059080B887
:100A9900E0700312398B9080D0E07003123BFC9018
:100AA9008000E07013301810122DBA906331EFF006
:100AB900D394004003120036908002E070069080C3
:100AC90000E06005D216020A14C216E4F51490611A
:100AD90004E06003020A14201C12906578E0600C9F
:100AE9007E0E7FE4122FB4E4906578F0301A12126A
:100AF900275B906331EFF0D394004005E0FF1200CB
:100B090032201903020C8A1225D4906331EFF07058
:100B190003020A14906375E054BF247F7003020B2B
:100B2900F3147003020BCB24026003020C2C201C6B
:100B3900077E0E7FEB122FB4202003020C8A9063EC
:100B49004DE07006906351E06067906682E0FF9027
:100B5900634DE0B50724906683E0FE90634EE0B5EF
:100B69000618906684E0FE90634FE0B5060C906627
:100B790085E0FE906350E06E6037906351E06F60EE
:100B890003020C8A906683E0FF906352E06F600372
:100B9900020C8A906684E0FF906353E06F60030261
:100BA9000C8A906685E0FF906354E06F6003020C45
:100BB9008AC2149065777401F0123F6C75120102B4
:100BC9000C8A90668BE060037401F090667AE0FF0E
:100BD900906377E06F6003020C8A90667AE004F014
:100BE900E4F512906575F0020C8A301403020C8A40
:100BF900906344E07003020A14906355740AF0127A
:100C09003D0BD214E4F512906575F090668604F0F8
:100C1900E4906679F0A3F0201C677E0E7FF9122F0D
:100C2900B4805E90668BE060037401F030145290DA
:100C39006375E020E74B906377E0FF906679E0FE0B
:100C49006F600D906681E07007EE146F703380134A
:100C5900906679E004F0906331E0FFD39404400397
:100C69001234AB9060007482F0A37401F090637742
:100C7900E0906002F07E607F007D031236F8020A80
:100C890014201403020DA2E5127068123ADEEF6017
:100C9900237E647F75906476E02404FD1236F89013
:100CA9006681E07009906355E0F512020A14E4F5D3
:100CB90012020A14906686E0D3943C40369066810D
:100CC900E0703090668604F0123258E4906475F052
:100CD900A37412F090667AE0906477F0A374FDF043
:100CE90090610563A20190647963A2017F12121FCA
:100CF900C1809E123F618F4DE54DB4011590600092
:100D09007483F0E4A3F07E607F007D021236F8025E
:100D19000A14E54DD39401401C9060007483F0A33C
:100D29007401F0E54D24FEA3F07E607F007D03127F
:100D390036F8020A14E51264016003020A14906588
:100D490075E004F0201C077E0F7F03122FB4906317
:100D590055E0C394C85004E02432F0906575E0C3AF
:100D69009405400DC214E4906577F0123F6C020AB5
:100D7900147C667D82906349E0FAA3E0FB7F02124E
:100D890038897E647F75906476E02404FD1236F814
:100D9900906355E0F512020A14E51264016003023A
:100DA9000A14906577E014604624FE6042147003CB
:100DB900020E9524046003020A14E4F5142020139A
:100DC9009065777404F0906575E05401F07512012F
:100DD900020A149080027410F0E4906577F090652F
:100DE9007504F07512FA90668274FFF0020A149085
:100DF9006682E07003020E7F9064757480F09064DF
:100E0900777401F0E4A3F0A304F0A37430F0A374A1
:100E19007BF0E4F54D747C254DF582E43464F5836B
:100E2900747DF0747D254DF582E43464F583E4F036
:100E3900E54D2407906476F07C667D82906349E0F5
:100E4900FAA3E0FB7F021238897E647F75E54D24A1
:100E590009FD1236F8906681E0601B123D0BD21431
:100E6900E4F512906575F090668604F0E490667971
:100E7900F0A3F0020A14302007E4906577F08006A9
:100E89009065777404F07512FA020A14908002745E
:100E990010F0751205906575E06401FFF0906577B3
:100EA9007401F0EF7019906351E06013FCA3E0FD49
:100EB900A3E0FEA3E0FF906682121B54020A14907D
:100EC900634DE0FCA3E0FDA3E0FEA3E0FF90668292
:090ED900121B54020A1480FE22CF
:10003600906376E0B444047F0180027F009063758C
:10004600E0B447047E0180027E00EE5F604A906362
:100056003EE0906377F090633FE0906378F09063C2
:1000660040E0906379F0906341E090637AF09063AA
:1000760042E090637BF0906343E090637CF0906392
:10008600767452F09062AE63A2019080A863A201DA
:100096007F06121FC102086F906331E0C3940850B7
:1000A6000302087890633EE0FF906377E06F600399
:1000B60002087890633FE0FF906378E06F60030288
:1000C6000878906340E0FF906379E06F6003020870
:1000D60078906341E0FF90637AE06F6003020878EE
:1000E600906342E0FF90637BE06F600302087890C4
:1000F6006343E0FF90637CE06F60030208789063DF
:1001060076E06444701A9080A8E0B4FF139062AE63
:1001160063A2019080A863A2017F06121FC180100E
:100126009062B2E09080ACF09062B3E09080ADF067
:1001360090668BE060037401F090668C7464F090B6
:1001460063767452F0906375E0646D600302027921
:100156007BFF7A0F790E12138A7BFF7A0F7928902C
:10016600633EE0F556A3E0F557A3E0F558A3E0F5A6
:1001760059A3E0F55AA3E0F55B12138A7556FF758D
:10018600570F7558857559FF755A0F755B917BFF2B
:100196007A0F795E12138A7BFF7A0F799A12138A85
:1001A6007BFF7A10790012138A7BFF7A10792D90E3
:1001B6006344E0F556A3E0F557A3E0F558A3E0F550
:1001C6005912138A7BFF7A10795790634DE0F556E2
:1001D600A3E0F557A3E0F558A3E0F55912138A7B7F
:1001E600FF7A107985906351E0F556A3E0F557A3A1
:1001F600E0F558A3E0F55912138A7BFF7A1079B31C
:1002060090633AE0F556A3E0F557A3E0F558A3E06E
:10021600F55912138A7BFF7A1079D6906336E0F58A
:1002260056A3E0F557A3E0F558A3E0F55912138A53
:100236007BFF7A1079F312138A7BFF7A11791CA25D
:1002460020E433F55612138A7BFF7A11794C9066B7
:1002560081E0F55612138A7BFF7A11797790668BC7
:10026600E0F55612138A122EBE7BFF7A1179AA1276
:10027600138A22906375E0644C70737E117FB0FB25
:10028600FDFC122CB390637DE0F54EA3E0F54FE440
:10029600F551E54E90637FF0A3E54FF07E117FEBBD
:1002A6007C637D7F7B02122CB3E4F550854F8285FB
:1002B6004E83E0FF747F2550F582E43463F583EFC7
:1002C600F0054FE54F7002054E0550E550B410DCC1
:1002D6007E117FEE7C637D7F7B10122CB30551E58A
:1002E60051C3941040AC7E117FF1122FB42290635B
:1002F60075E0646C7060F5527E117FF3FBFDFC12B5
:100306002CB3E4F551E490637FF0A3E552F07E113F
:100316007FEB7C637D7F7B02122CB3E4F550A85201
:10032600E6FF747F2550F582E43463F583EFF0052C
:10033600520550E550B410E67E117FEE7C637D7F5A
:100346007B10122CB30551E551C3940840B77E11BA
:100356007FF1122FB422906375E0644B7061F55003
:1003660074672550F582E43463F583E06032746780
:100376002550F582E43463F583E0F4602374672541
:1003860050F582E43463F583E0FF747D2550F582F1
:10039600E43463F583E0B507100550E550B408C0B2
:1003A6009061047432F002086F9063757421F03026
:1003B6001C0302086F7E127F2E122FB402086F9064
:1003C6006375E0B4521A201C077E127F36122FB4D2
:1003D6009063757472F07E637F757D0812367122A4
:1003E600906375E064497045201C077E127F4112B8
:1003F6002FB490637DE0F54EA3E0F54FE4F550850C
:100406004F82854E83E0FF747F2550F582E4346386
:10041600F583EFF0054FE54F7002054E0550E550A8
:10042600B480DC7E637F757D8A1236712290637597
:10043600E064437046201C077E127F49122FB49059
:10044600637DE0F54EA3E0F54FE4F550854F8285D8
:100456004E83E493FF747F2550F582E43463F5837D
:10046600EFF0054FE54F7002054E0550E550B4809C
:10047600DB7E637F757D8A12367122906375E06438
:100486005A7053201C077E127F52122FB490637D40
:10049600E0F54EA3E0F54F7C637D7F7B80AF4FAEEA
:1004A6004E123E0FE4F550854F82854E83E493FF4E
:1004B600747F2550F582E43463F583EFF0054FE54C
:1004C6004F7002054E0550E550B480DB7E637F75A4
:1004D6007D8A12367122906375E0644460030205DA
:1004E6006D90637DE0FF6444700302086FEFB431E2
:1004F6000CC21C7E127F5E122FB402086F90637DC1
:10050600E0B4300CD21C7E127F6A122FB402086F40
:1005160090637DE0B4320CD21D7E127F77122FB429
:1005260002086F90637DE0B4330CC21D7E127F8596
:10053600122FB402086F90637DE0B4340CD21E7E95
:10054600127F94122FB402086F90637DE0B4350CCD
:10055600C21E7E127FA1122FB402086F90637DE047
:10056600FF12001E02086F906104E07013201C0742
:100576007E127FAF122FB49063757421F002086F5C
:100586009061047432F0906375E0FFB45104C2AF19
:1005960080FEEF64577045201C077E127FBD122F28
:1005A600B490637EE0906331F0E4F550906331E0FF
:1005B600FFE550C39F400302086F747F2550F58204
:1005C600E43463F583E0FF90637DE0255024ADF5C8
:1005D60082E43461F583EFF0055080D0906375E0D6
:1005E60064536003020690201C077E127FC8122FF8
:1005F600B490633EE0FF9061B6E06F703C90633F5D
:10060600E0FF9061B7E06F7030906340E0FF90616B
:10061600B8E0B50724906341E0FF9061B9E0B50703
:1006260018906342E0FF9061BAE0B5070C9063430F
:10063600E0FF9061BBE06F60169063757421F03047
:100646001C0302086F7E127FD7122FB402086FE4D4
:10065600F550E4F515AF50FE74AD2550F582E4343F
:1006660061F583E0FD123E6A0550E550C394FE40F5
:10067600E1C2AFE4907FF0F0A3F0907FFD74AAF0A2
:10068600A374FFF0A37455F080FE906375E0644F89
:10069600704C90637DE0F54EA3E0F54FE54F454E77
:1006A600700A201C077E127FE0122FB4201C077EE2
:1006B600127FE7122FB4E4F550747F2550F582E4DB
:1006C6003463F583E0854F82854E83F0054FE54F11
:1006D6007002054E0550E550B480DE02086F906347
:1006E60075E0FFB4452190637DE0FDA3E0907FF0C7
:1006F600CDF0A3EDF0C2AF907FFD74AAF0A374FF16
:10070600F0A37455F080FEEF6465600302087890EC
:10071600637DE0FFA3E0907FF0CFF0A3EFF0E4F578
:100726004EF54FD3907FF1E0954F907FF0E0954ED8
:100736004020E4F515254FFFE54E3401FE854F8236
:10074600854E83E0FD123E6A054FE54F7002054E69
:1007560080D17E127FE912377FEF4E6020120003B0
:10076600906344EFF0120003906345EFF01200032C
:10077600906346EFF0120003906347EFF07E127F1E
:10078600EF12377FEF4E602012000390634DEFF0BB
:1007960012000390634EEFF012000390634FEFF0E8
:1007A600120003906350EFF07E127FF512377FEF51
:1007B6004E6020120003906351EFF0120003906325
:1007C60052EFF0120003906353EFF01200039063B0
:1007D60054EFF07E127FFB12377FEF4E602012003F
:1007E6000390633AEFF012000390633BEFF01200C0
:1007F6000390633CEFF012000390633DEFF07E132D
:100806007F0112377FEF4E6020120003906336EFB0
:10081600F0120003906337EFF0120003906338EF95
:10082600F0120003906339EFF0E4F550E4F515E5B6
:10083600502401FFE433FE74362550F582E4346318
:10084600F583E0FD123E6A0550E550C3944340DC53
:10085600C2AFE4907FF0F0A3F0907FFD74AAF0A3FE
:1008660074FFF0A37455F080FE7E637F757D0812D9
:03087600367122B6
:103DD700AE07EEC39430400BEED394395005EE2472
:103DE700D0FF22EEC39461400BEED394665005EEEC
:103DF70024A9FF22EEC39441400BEED3944650050D
:083E0700EE24C9FF22AF0622E0
:103F2C009062ADE004F070069062ACE004F0906238
:0A3F3C00ACE0FEA3E0FF123ED62227
:10000300123F2C123DD7EFC454F0FEC006123F2C12
:08001300123DD7D0E02FFF22BF
:103B9F00E4906CC0F0123F2C906CC1EFF0C39430E6
:103BAF004018E0FFD394395011906CC0E02405F514
:103BBF0082E43461F583EFF08011906CC0E024054E
:103BCF00F582E43461F583E4F0800C906CC0E0047E
:103BDF00F0E0D3940840BE755A00755B00755C0029
:0D3BEF00E4F55D7B017A6179051222A122C7
:10377F008E538F549062ACE4F0A374FFF0123F2C81
:10378F00EF606EF4606B855482855383E493B507C5
:10379F00EC755501E5542555F582E43553F583E471
:1037AF009360259062ADE02555FF9062ACE0340048
:1037BF00FE123ED6E5542555F582E43553F583E4E4
:1037CF0093B50704055580CCE5542555F582E435AE
:1037DF0053F583E49370A6E55524FFFFE434FFFE11
:1037EF009062ADE02FF09062ACE03EF07E007F0182
:0537FF0022E4FEFF22A0
:103331007E137F0712377FEF4E70037F01227E13CA
:103341007F0A12377FEF4E600C123F2CEF24D024FE
:10335100FF92208002D2207E137F1012377FEF4E22
:10336100600C123F2CEF24D0906681F08005E49030
:103371006681F07E137F1612377FEF4E600C123F8D
:103381002CEF24D090668BF08005E490668BF07E64
:10339100137F1C12377FEF4E600C123F2CEF24D0AD
:1033A10024FF92128002C21290633E63A2019066D2
:1033B1007B63A2017F06121FC130123B7E137F2265
:1033C10012377FEF4E603012000390667BEFF012F0
:1033D100000390667CEFF012000390667DEFF0121F
:1033E100000390667EEFF012000390667FEFF0120B
:0A33F1000003906680EFF07F0022D9
:103D5500906576E0C3947C40027F0A906576E0FE2C
:103D650004F074B42EF582E43462F583EFF0BF0AF3
:103D750027906576E0FF04F074B42FF582E4346291
:103D8500F583E4F0906576E0FF123804906576746B
:093D950008F09062B5E004F02290
:103C58009080007480F090633663A201F583F5824A
:103C680063A2017F08121FC190633E63A201908086
:103C78008863A2017F0A121FC19080927407F0A383
:103C880074D0F0A37406F0906348E0FF9080B1F020
:103C98009080E1EFF09080957455F0A3F09080004B
:0A3CA8007401F090800974F0F0221E
:103A0500908009E04410F09080A0E070609080A163
:103A15007482F09080A874FFF0A3F0A3F0A3F07F68
:103A2500039080AEEFF0A374CBF09080007402F0A9
:103A3500906CB0121B6000000000906CB0E09080AC
:103A450040F0906CB1E0908041F0906CB2E09080D5
:103A550042F0906CB3E0908043F0A3E4F0A3F0A3B0
:0E3A6500F0A3F0908018F0A3F0A3F0A3F022DD
:103BFC00908009E04440F09080D17482F07F039073
:103C0C0080DEEFF0A374CCF09080027402F0906C24
:103C1C00B4121B6000000000906CB4E0908058F06F
:103C2C00906CB5E0908059F0906CB6E090805AF0B2
:103C3C00906CB7E090805BF0A3E4F0A3F0A3F0A34A
:0C3C4C00F0908030F0A3F0A3F0A3F02271
:10398B00908009E04420F09080B8E0706C9080B992
:10399B007482F07F039080C6EFF07FCDA3EFF07FB2
:1039AB00039080C4EFF0A374CDF09080C074FFF04F
:1039BB00A3F0A3F0A3F09080017402F0906CB81206
:1039CB001B6000000000906CB8E090804CF0906C95
:1039DB00B9E090804DF0906CBAE090804EF0906C16
:1039EB00BBE090804FF0A3E4F0A3F0A3F0A3F09022
:0A39FB008024F0A3F0A3F0A3F02253
:103889008C4E8D4FA907EAFDE975F018A424ACFF09
:10389900E5F034808F82F583EDF0EBFDE975F018E2
:1038A900A4FFAEF024ACFBEE34808B82F583A3ED4C
:1038B900F0854F828C83E0FDEF24A8FFEE3480FE73
:1038C9008F82F583EDF0854F828C83A3E08F828E02
:1038D90083A3F0854F82854E83A3A3E0FDE975F0AC
:1038E90018A424A8FFE5F03480FE8F82F583A3A3F2
:1038F900EDF0854F828C83A3A3A3E08F828E83A3EF
:04390900A3A3F02262
:103671008D53AB07AA06908000E030E5079065788E
:103681007401F022906CB0E0FCA3E0FDA3E0FEA386
:10369100E0F5578E568D558C54AE02AF038E838F55
:1036A1008263A201E556540744C0F58385578263BE
:1036B100A201AF53122033E4FCFDFEE5572553F57B
:1036C10057EE3556F556ED3555F555EC3554F5545F
:1036D100908040E554F0A3E555F0A3E556F0A3E54D
:1036E10057F09080007420F0AF57AE56AD55AC54F2
:0736F100906CB0121B542283
:1036F8008D4EAB07AA06908002E030E5079065780A
:103708007403F022906CB4E0FCA3E0FDA3E0FEA3F8
:10371800E0F5528E518D508C4FAE02AF038E838FE1
:103728008263A201E551540744D0F5838552826330
:10373800A201AF4E122033E4FCFDFEE552254EF502
:1037480052EE3551F551ED3550F550EC354FF54FFA
:10375800908058E54FF0A3E550F0A3E551F0A3E5BC
:1037680052F09080027420F0AF52AE51AD50AC4F81
:07377800906CB4121B5422F7
:1033FB008F4E908001E030E5099065787402F07F84
:10340B000022906CB8E0FCA3E0FDA3E0FEA3E0F586
:10341B00528E518D508C4F90667B63A201E55154B7
:10342B000744C8F58385528263A2017F06122049A7
:10343B00E5522406F552E43551F551E43550F5507B
:10344B00E4354FF54F90657963A201E5515407447C
:10345B00C8F58385528263A201AF4E122049E4FC6A
:10346B00FDFEE552254EF552EE3551F551ED355039
:10347B00F550EC354FF54F90804CE54FF0A3E550F0
:10348B00F0A3E551F0A3E552F09080017420F0AF6A
:10349B0052AE51AD50AC4F906CB8121B54AF4E2284
:102DBA009081E0E0F54E054E054E054E054E054E56
:102DCA00054E054E054E054E054E908010E0F55114
:102DDA00A3E0F552A3E0F553A3E0F5549081E1E0B6
:102DEA00F54E054E054E054E054E054E054E054E51
:102DFA00054E054E054E908014E0F555A3E0F556B4
:102E0A00A3E0F557A3E0F558E557B55308E558B5DB
:102E1A0054037F0022E4F54EE557540744E0F58356
:102E2A0085588263A20190637563A2017F0812200C
:102E3A007990637763A2019062AE63A2017F061262
:102E4A001FC1906375E0F54FA3E0F550E4F54E908D
:102E5A006375E0702AA3E024F8F54EE55754074459
:102E6A00E0F58385588274082582F582E43583F576
:102E7A008363A20190637563A201AF4E122079AEFB
:102E8A004FE4FCFDE5582550F558E5573EF557ED5A
:102E9A003556F556EC3555F555908014E555F0A3A1
:102EAA00E556F0A3E557F0A3E558F090800074408A
:042EBA00F0AF4E2205
:1025D4009081E6E0F54E054E054E054E054E054E3E
:1025E400054E054E054E054E054E908028E0F551EA
:1025F400A3E0F552A3E0F553A3E0F5549081E7E09E
:10260400F54E054E054E054E054E054E054E054E3E
:10261400054E054E054E90802CE0F555A3E0F55689
:10262400A3E0F557A3E0F558E4F54EE557B5530A92
:10263400E558B55405C219022740E557540744F03C
:10264400F58385588263A20190637563A2017F08B4
:10265400122079906375E0F54FA3E0F550E55045FD
:102664004F70099080027410F07F0022906682E01F
:10267400FFF46030906377E06F6003022707906691
:1026840083E0FF906378E06F7079906684E0FF9058
:102694006379E06F706D906685E0FF90637AE06F18
:1026A4006031805F906377E0906682F0906378E0B9
:1026B400906683F0906379E0906684F090637AE0AA
:1026C400906685F090637BE0FFA3E0906349CFF0D0
:1026D400A3EFF0906375E0702AA3E024F8F54EE5CB
:1026E40057540744F0F58385588274082582F5828F
:1026F400E43583F58363A20190637563A201AF4E51
:10270400122079AE4FE4FCFDE5582550F558E55705
:102714003EF557ED3556F556EC3555F555AF54AEF7
:1027240053AD52AC51AB58AA57A956A855D3121B56
:102734003040099080027410F07F002290802CE5D4
:1027440055F0A3E556F0A3E557F0A3E558F09080C3
:07275400027440F0AF4E22B9
:10275B009081E3E0F54E054E054E054E054E054EB8
:10276B00054E054E054E054E054E90801CE0F5516D
:10277B00A3E0F552A3E0F553A3E0F5549081E4E018
:10278B00F54E054E054E054E054E054E054E054EB6
:10279B00054E054E054E908020E0F555A3E0F5560D
:1027AB00A3E0F557A3E0F558E4F54EE557B5530A0A
:1027BB00E558B55405C21A0228B1E557540744E849
:1027CB00F58385588263A20190600463A2017F0E9A
:1027DB0012208F906004E0F54FA3E0F55090600C51
:1027EB00E0FFF4604A90667BE0FEEF6E7079A3E049
:1027FB00FF90600DE06F706F90667DE0FF90600E54
:10280B00E06F706390667EE0FF90600FE06F705733
:10281B0090667FE0FF906010E06F704B906680E0F9
:10282B00FF906011E06F703FE4906013F0800890B0
:10283B00601374FFF0D2D9906004E0702AA3E024F7
:10284B00F2F54EE557540744E8F583855882740E2C
:10285B002582F582E43583F58363A20190600463DE
:10286B00A201AF4E12208FAE4FE4FCFDE558255070
:10287B00F558E5573EF557ED3556F556EC3555F50C
:10288B0055AF54AE53AD52AC51AB58AA57A956A83D
:10289B0055D3121B305006E550454F7009908001FF
:1028AB007410F07F0022908020E555F0A3E556F0E0
:1028BB00A3E557F0A3E558F09080017440F0AF4EBC
:0128CB0022EA
:102FB4008E538F54908000E030E50790657874015B
:102FC400F022906CB0E0FCA3E0FDA3E0FEA3E0F5EA
:102FD4005A8E598D588C57E55AFFE5595407FEE42B
:102FE4002FF556EE34C0F555855682F5837423F0DB
:102FF4000556E556700205555355C7F58285558328
:10300400740AF00556E556700205555355C790638A
:103014003E63A20185558385568263A2017F061211
:10302400203374062556F556E43555F555855383F6
:1030340085548263A20185558385568263A2011259
:103044002017E4FCFDFE906CB0E0F8A3E0F9A3E0E7
:10305400FAA3E02FFFEE3AFEED39FDEC38FCEF2445
:1030640008FFE43EFEE43DFDE43CFC906CB0121B22
:1030740054906CB0E0908040F0906CB1E09080414E
:10308400F0906CB2E0908042F0906CB3E09080439A
:08309400F09080007420F0228E
:102CB3008E538F548C558D568B57908000E030E5A2
:102CC300079065787401F022906CB0E0FCA3E0FDFE
:102CD300A3E0FEA3E0F55D8E5C8D5B8C5AE55DFFA2
:102CE300E55C5407FEE42FF559EE34C0F5588559D9
:102CF30082F5837423F00559E5597002055853583A
:102D0300C7F582855883740AF00559E559700205A1
:102D1300585358C790633E63A201855883855982EF
:102D230063A2017F0612203374062559F559E43551
:102D330058F55885538385548263A201855883854A
:102D4300598263A2011220178F5EEF2559F559E4CA
:102D53003558F558E557601785558385568263A224
:102D63000185588385598263A201AF57122033E549
:102D73005E24082557F557FFE4FCFDFEE55D2FF5BE
:102D83005DEE355CF55CED355BF55BEC355AF55A7C
:102D9300908040E55AF0A3E55BF0A3E55CF0A3E582
:102DA3005DF09080007420F0AF5DAE5CAD5BAC5A1B
:072DB300906CB0121B5422CA
:10317D008E4E8F4F8D50908000E030E50790657832
:10318D007401F022906CB0E0FCA3E0FDA3E0FEA37F
:10319D00E0F5568E558D548C53E556FFE555540785
:1031AD00FEE42FF552EE34C0F551855282F583744D
:1031BD0023F00552E552700205515351C7F5828532
:1031CD005183EBF00552E552700205515351C790F2
:1031DD00633E63A20185518385528263A2017F06FE
:1031ED0012203374062552F552E43551F551854EB2
:1031FD0083854F8263A20185518385528263A2012B
:10320D00AF5012203374082550F550FFE4FCFDFE3D
:10321D00E5562FF556EE3555F555ED3554F554EC7F
:10322D003553F553908040E553F0A3E554F0A3E5F5
:10323D0055F0A3E556F09080007420F0AF56AE55D2
:0B324D00AD54AC53906CB0121B542227
:103804008F67908000E030E5079065787401F022BE
:10381400906CB0E0FCA3E0FDA3E0FEA3E0F56B8EAA
:103824006A8D698C68E56BFFE56A5407FEE42FFF37
:10383400EE34C09062B463A201F5838F8263A20167
:10384400AF67122033E4FCFDFEE56B2567F56BEEF4
:10385400356AF56AED3569F569EC3568F568908087
:1038640040E568F0A3E569F0A3E56AF0A3E56BF031
:103874009080007420F0AF6BAE6AAD69AC68906C58
:05388400B0121B5422EC
:10309C008E4E8F4FAB05908000E030E50790657841
:1030AC007401F022906CB0E0FCA3E0FDA3E0FEA361
:1030BC00E0F5558E548D538C52E555FFE55454076D
:1030CC00FEE42FF551EE34C0F550855182F5837432
:1030DC0023F00551E551700205505350C7F5828518
:1030EC005083EBF00551E5517002055090633E633F
:1030FC00A20185508385518263A2017F0612203381
:10310C0074062551F551E43550F5505350C7E54E32
:10311C00855182855083F00551E55170020550535D
:10312C0050C7F582855083E54FF00551E55170028B
:10313C0005505350C7E555240AF555E43554F5545C
:10314C00E43553F553E43552F552908040E552F096
:10315C00A3E553F0A3E554F0A3E555F0908000747B
:10316C0020F0AF55AE54AD53AC52906CB0121B5412
:01317C002230
:0B3F5600E4FEEEC39F50030E80F82233
:103ED600A2AF9221C2AF438E2075D2028F828E830B
:0D3EE600E0FFE4F5D2538EDFA22192AF225F
:103E6A00E5D220E0FBA2AF9221C2AF43D2028F82F9
:103E7A008E83EDF075D25063D250A22192AFE5D273
:043E8A0020E0FB2217
:10390D00E4FDED2401FFE433FE123ED674362DF5B1
:10391D0082E43463F583EFF00DBD3FE6E4FDED2465
:10392D007FFFE433FE123ED6742D2DF582E4346113
:10393D00F583EFF0742D2DF582E43461F583E0709D
:10394D001B742D2DF582E43461F5837420F0742EF3
:10395D002DF582E43461F583E4F080040DBD80BE65
:10396D00E49061ACF0FDEDFF7E00123ED674AD2DFE
:0E397D00F582E43461F583EFF00DBDFEE92222
:103E0F008B53A2AF9221C2AF85A25453A2FE8E83D1
:103E1F008F8205A28C838D8274091220BDE55353C6
:103E2F00A2FE43A2201220BF53A2DF8554A2A221DB
:043E3F0092AFFF221D
:103EF300A2AF9221C2AF8C838D82EF1220BD43A269
:0D3F0300201220BF53A2DFA22192AFFF22A7
:103E8E008F4EA2AF9221C2AFE4F5838D82740612DB
:103E9E0020BDE54E43A2201220BF53A2DFA22192E5
:043EAE00AF7F0122BF
:103EB2008F4EA2AF9221C2AFE4F5838D82740A12B3
:103EC20020BDE54E43A2201220BF53A2DFA22192C1
:043ED200AF7F01229B
:101EE600A907E7FFA805EF93C3966008403B74FC7B
:101EF6002FFF80F00F08EF93C3966008402B74FB0A
:101F06002FFF80E00F08EF93C3966008401B74FA1A
:101F16002FFF80D00F08EF93D3966008400B74F91B
:101F26002FFF80C01F1F1F1F1FEF54FEF80303F76C
:101F3600E893FC08E893FD08E893FE08E893FF227F
:101F460009E993C39D6008402974FB29F980F109CA
:101F5600E993C39E6008401A74FA29F980E209E9F8
:101F660093D39F6008400B74F929F980D319191986
:101F76001919E9C313C313FF22740093F8ECC3982D
:101F86004024701F740193F8EDC3984019701474BF
:101F96000293F8EEC398400E7009740393F8EFC3EA
:101FA6009840037F00227F0122EDF8E6F008A3DFC8
:101FB600FA22EDF8E0F608A3DFFA22E0A363A20115
:101FC600F0A363A201DFF475A2002263A201F0A3CD
:101FD60063A20122E0A363A201F0A363A201E0A32E
:101FE60063A201F0A363A201E463A201F0A363A2CA
:101FF60001DFE175A20022E0A363A2016DFE936CEE
:10200600FDEE058393FC158363A201DFEA75A2004A
:10201600227F00E493A363A201F00F600CA3E58383
:10202600C2E3F58363A20180EA75A20022E0A363FE
:10203600A201F0A3E583C2E3F58363A201DFEE7597
:10204600A20022E0A363A201F0A3E583C2E4D2E3E7
:10205600F58363A201DFEC75A20022E0A363A2016F
:10206600F0A3E58344F8C2E5F58363A201DFEC75CE
:10207600A20022E583C2E3F583E0A363A201F0A3F5
:1020860063A201DFEE75A20022E583C2E4D2E3F586
:1020960083E0A363A201F0A363A201DFEC75A200B3
:1020A60022E58344F8F583E0A363A201F0A363A2CB
:1020B60001DFEE75A20022F922C002C004C006129A
:0920C600FFF0D006D004D0022284
:10001E00BF360BD207E4F526F527F546F547BF3771
:04002E0002C20722E1
:103B4100C2A9438902906CABE0FFF58C8F8A75D9CD
:103B51000475DA4875DB3175DC4975DD4975DE318F
:103B6100E4F5E9F5F9F5EBF5FB906CA9E060167564
:103B7100EC1075ED10E4F5FCF5FD754208753C108F
:103B8100754101801375EC8075ED80E4F5FCF5FD60
:0E3B9100754280F53C754110E4F5EEF5FE221C
:103D9E00E4FEAF8CEFFD906CAAE07003A3E06D60C3
:103DAE0005123B417E01E5D920E2057E02123B4120
:103DBE00E58920E105123B417E03D28C75D8407512
:093DCE00B740D2AED2AFAF06221D
:030033000220CFD9
:1020CF00C0E0C0F0C083C082C0D075D008C2AF30AE
:1020DF00DC56C3E5EC95EEC395425012E54125EC75
:1020EF00F5EC30D70405FC801685FCFC8011C3E5A8
:1020FF00EC9541F5EC30D70415FC800385FCFC30E2
:10210F000724852782852683E590F00527E527702C
:10211F00020526F582852683E5EEF00527E5277073
:10212F0002052653260FC2DC30D929300724852714
:10213F0082852683E590F00527E52770020526F5B1
:10214F0082852683E5EBF00527E5277002052653E8
:10215F00260FC2D920DA03022220E53C700405FCC9
:10216F008010E53C25ECF5EC30D70405FC800385A9
:10217F00FCFC20080302221E302A41AF40AE3FADC7
:10218F003EAC3D7801121B418F408E3F8D3E8C3D02
:10219F00309712E540F540E53FF53FE53EF53EE56A
:1021AF003D4480F53D200627E540F540E53FF53FEE
:1021BF00E53EF53EE53D6480F53D8013E528C3130C
:1021CF00F5283097042480F52820060363288030F3
:1021DF002A23E4FFE53FFEE53EFDE53DFCAB4BAAC0
:1021EF004AA949A848C3121B307024F543F53AF5A4
:1021FF0028C22A801A0543E5435407701253433F00
:10220F00E543131313541F242AF8A628752800C278
:10221F00DA30DB71E53C700405FD8010E53C25EDFF
:10222F00F5ED30D70405FD800385FDFDE544653BE5
:10223F006029E53B54077013E53B131313541F2418
:10224F0032F8E6F5292004036329FFE52913929656
:10225F00E529C313F529053B533B3FB292300723C2
:10226F00852782852683E590F00527E527700205EF
:10227F0026F582852683E4F00527E52770020526DB
:10228F0053260FC2DBD2AFD0D0D082D083D0F0D0C4
:02229F00E0322B
:101C80004241554400494E565F52454300494E5625
:101C90005F5452414E5300494E565F414C4C0044F4
:101CA0004543495F56414C00003E2A2C312CCFE081
:101CB000F0E0ECE5F2F0FB20F1E8EDF5F0EEEDED13
:101CC000EEE3EE20EFEEF0F2E00A003E4C2C423064
:101CD000312C256C752CD1EAEEF0EEF1F2FC20EE01
:101CE000E1ECE5EDE02C35302C3130302C32303069
:101CF0002C3330302C3630302C313230302C3234E2
:101D000030302C343830300A003E422C4731302CF1
:101D10002562752CC8EDE2E5F0F1E8FF20EDE0204A
:101D2000EFF0E8B8ECE50A003E422C4731312C25B3
:101D300062752CC8EDE2E5F0F1E8FF20EDE020EF60
:101D4000E5F0E5E4E0F7E50A003E422C4730322CAE
:101D50002562752CD3EFF0E0E2EBE5EDE8E520EF4E
:101D6000EEF2EEEAEEEC2020285254532D43545369
:101D7000290A003E532C4730332C256C752CC7E0C4
:101D8000E4E5F0E6EAE020F1F2E0F0F2E020EFE551
:101D9000F0E5E4E0F7E828ECF1290A003E532C478F
:101DA00030332C256C752C202AE7E0E4E5F0E6EAD8
:101DB000E020F1F2E0F0F2E020EFE5F0E5E4E0F71A
:101DC000E828ECF1290A003E2A2C312CC0E4E0EF8F
:101DD000F2E5F020F1E8EDF5F0EEEDEDEEE3EE20CA
:101DE000EAE0EDE0EBE02E20CFF0EEF2EEEAEEEBF3
:101DF00020D0CFD22D383028C0E8F1F2290A003E99
:101E0000532C5230312C256C752CCFE0F0E0ECE5F2
:101E1000F2F0FB20EFF0EEF0E5E6E8E2E0EDE8FFBF
:101E200020D6C1C80A003C21003C4230313D003C74
:101E30004731303D003C4731313D003C4730323D79
:101E4000003C4730333D003C5230313D000A456D87
:101E50007074792120000A54726961646520200041
:101E60000A526563206572726F7221000A526563BF
:101E70002064617461000A52656320424349210075
:101E80000A526563656976656420466C6167212046
:101E9000000A5472616E736D697420000A54726195
:101EA0006E736D697420666C61670A00FF1C80FFA9
:101EB0001C85FF1C8DFF1C97FF1C9FFF1CA80008A2
:101EC000040C020A060E0109050D030B070F0001A1
:101ED00001000100000101000001000101000102F8
:061EE0000407080B0D0EC3
:103F160052668D0000000000000000000000000056
:053F2600000000000096
:0100320022AB
:103CB2008F57906AA7E0FF04F074A92FF582E434CD
:103CC20066F5837420F0E4FFEFC39D503BE5577522
:103CD200F003A424ACF582E4341EF583E493FB7470
:103CE2000193FA740293F98F827583001219F3FE1D
:103CF200906AA7E024A9F582E43466F583EEF00F1A
:093D0200906AA7E004F080C022E1
:103E4300742D2FF582E43461F583E0FE642060165F
:103E5300906AA7E0FD04F074A92DF582E43466F5B9
:073E630083EEF00F80DA226C
:10244500E4906AA7F0F54FE54F75F003A424ACF5C9
:1024550082E4341EF583E493FB740193FA740293CA
:10246500F91219DA70030225D3E4F551F552F55046
:10247500742D2550F582E43461F583E0FF70030285
:1024850025CEE54F75F003A424ACF582E4341EF5A2
:1024950083E493FB740193FA740293F98551827571
:1024A50083001219F3FEEFB50608755201055102B6
:1024B50025C9E55270030225C9EE60030225C4ADA6
:1024C50051AF4F123CB2E54F1470030225861470CC
:1024D5000302258A14700302258E147003022594C5
:1024E500240460030225CEAF50123E43742D2550BF
:1024F500F9E43461FA7B01C0031B8B5A755B0075E7
:102505005C00E4F55DD0031222A18F568E558D54E3
:102515008C53E4FFFEFDFCAB56AA55A954A853C342
:10252500121B306022AB56AA55A954A853E47F204C
:102535007E1CFDFC121A90121B22906CAAEEF0A3D1
:10254500EFF0E4906CA9F0E47FB07E04FDFCAB569F
:10255500AA55A954A853D3121B30406D906CA97489
:1025650001F0AB56AA55A954A8537F007EC2FD7C45
:1025750000121A90121B22906CAAEEF0A3EFF080C5
:1025850048D2068044D2048040D206D204803AAFB5
:1025950050123E43742D2550F9E43461FA7B01C095
:1025A500031B8B5A755B00755C00E4F55DD0031267
:1025B50022A18F568E558D548C5385567D800AE405
:0F25C500F552F5510550022475054F02244C22A2
:102EBE007BFF7A1C79A912138A906CA9E0602FA36C
:102ECE00E0FEA3E0FFC3E49FFFE49EFEAB07FAE43F
:102EDE00F9F8FF7EC27D01FC121A908F598E588D23
:102EEE00578C567BFF7A1C79CB12138A802F906CED
:102EFE00AAE0FEA3E0FFC3E49FFFE49EFEAB07FA49
:102F0E00E4F9F87F207E1CFDFC121A908F598E5822
:102F1E008D578C567BFF7A1C79CB12138A7BFF7AE6
:102F2E001D7909A206E433F55612138A7BFF7A1D2A
:102F3E007928A204E433F55612138A7BFF7A1D79A1
:102F4E0049A20AE433F55612138A300A1F7BFF7A20
:102F5E001D79739066A1E075F00AA4FFAEF0E48FC0
:102F6E00598E58F557F55612138A801D7BFF7A1D20
:102F7E00799C9066A1E075F00AA4FFAEF0E48F593B
:102F8E008E58F557F55612138A7BFF7A1D79C712A4
:102F9E00138A7BFF7A1D79FFE4857D59F558F55725
:062FAE00F55612138A2201
:102B77007E1E7F2612377FEF4E70037F01227E1E57
:102B87007F2912377FEF4E7003022C1E123B9F9056
:102B97006CBC121B54E4FFFEFDFC906CBCE0F8A378
:102BA700E0F9A3E0FAA3E0FBC3121B306025906CA9
:102BB700BCE0F8A3E0A3E0A3E0E47F207E1CFDFCDB
:102BC700121A90121B22906CAAEEF0A3EFF0E49079
:102BD7006CA9F0E47FB07E04FDFC906CBCE0F8A328
:102BE700E0F9A3E0FAA3E0FBD3121B304038906C66
:102BF700A97401F0906CBCE0F8A3E0A3E0A3E07F28
:102C0700007EC27D017C00121A90121B22906CAAD2
:102C1700EEF0A3EFF0800F906CAA74FFF0A374B8E6
:102C2700F0E4906CA9F07E1E7F2F12377FEF4E6085
:102C37000C123F2CEF24D024FF92068002C2067E9E
:102C47001E7F3512377FEF4E600C123F2CEF24D0DA
:102C570024FF92048002C2047E1E7F3B12377FEF5F
:102C67004E600C123F2CEF24D024FF920A8002C240
:102C77000A7E1E7F4112377FEF4E6013123B9FE49F
:102C87007B0AFAF9F8121A909066A1EFF08005E432
:102C97009066A1F07E1E7F4712377FEF4E600712C6
:0C2CA7003B9F8F7D8003757D027F002223
:103ADE00300E5D30102FC210E4906475F0906CA81B
:103AEE00E004FF906476F090667AE0906477F0A33D
:103AFE007410F09067AA63A20190647963A2011218
:103B0E001FC17F0122E4906475F0A3E579F0906601
:103B1E007AE0906477F0A37403F09069A163A20138
:103B2E0090647963A201AF79121FC1C20E7F012288
:033B3E007F0022E3
:1034AB008F4E906378E06410702A7F797583630583
:1034BB008263A2019068A763A201E54E24FCFF1270
:1034CB001FC1D201E54E24FCF576E4F57BF56D7555
:1034DB0074FE8073E54E24FCFFC313F54E754F0449
:1034EB00E4F550E550C3954E505DAF4F054F7475E5
:1034FB002FF582E43463F583E075F002A424A8F978
:10350B00746A35F0FA9068A47401F0A3EAF0A3E9A9
:10351B00F09068A4E0FBA3E0FAA3E0F97440121A60
:10352B0020AF4F054F74752FF582E43463F583E0BC
:10353B00FF9068A4E0FBA3E0FAA3E0F9900001EF91
:0A354B00121A320550809CD20D22A6
:103A7300906CAA74FFF0A374B8F0E4906CA9F09072
:103A83006AA7F0D22AF540F53FF53EF53DF54B75B3
:103A93004A66754996754899C203C208C20EC20C9C
:103AA300C20D757D02122B77EF6003122445E4F5F6
:103AB3004EE54E75F002A424A8F9746A35F0FA7B3A
:103AC300019068A4EBF0A3EAF0A3E9F0E4121A2052
:0B3AD300054EE54EB4FADA123B41222A
:103D0B00C203D208C20ED22AE4F540F53FF53EF5C8
:103D1B003DF54B754A6675499675489990668F12B5
:103D2B001B6000000000906693121B6000000000F7
:103D3B00906697121B600000000090669B121B6040
:0A3D4B0000000000123D9E8F4E2282
:10325800E4FF0F2405F582E43461F5837408F00F68
:1032680074052401F582E43461F583E4F0754E01B8
:10327800754F66755092FEAB4EE5501550AA4F70CB
:1032880002154FF91219DAFDAC070F74052CF582F7
:10329800E43461F583EDF00EBE04DC754E01754F24
:1032A80066755096E4FEAB4EE5501550AA4F700275
:1032B800154FF91219DAFDAC070F74052CF582E4E5
:1032C8003461F583EDF00EBE04DC754E01754F6672
:1032D80075509AE4FEAB4EE5501550AA4F70021592
:1032E8004FF91219DAFDAC070F74052CF582E43496
:1032F80061F583EDF00EBE04DC754E01754F667501
:10330800509EE4FEAB4EE5501550AA4F7002154F83
:10331800F91219DAFDAC070F74052CF582E4346153
:09332800F583EDF00EBE04DC2279
:1028CC008D4E8B4F8A508951E4F552EF54E0FEC483
:1028DC00135407901EDE93FEC454F04252EF541C66
:1028EC00FE1313543F9342520551E55170020550AB
:1028FC0014F9E552121A20E55254C0FEC4540F903C
:10290C001ECE93FEE552540C93FDEE2DF553E5527D
:10291C0054A0FEC4540F93FEE552540A93FDEE2DC1
:10292C00F554E4F552EF540325E0FFE433FEE54E95
:10293C005480FDC41313135401FDEEEF4D24DEF54A
:10294C0082741E3EF583E493FFC454F04252E54E6C
:10295C005470FFC4540F901EDE934252AB4F05517E
:10296C00E551AA507002055014F9E552121A20E5EF
:10297C005254C0FFC4540F901ECE93FFE552540C1A
:10298C0093FEEF2E2553F553E55254A0FFC4540F7C
:10299C0093FFE552540A93FEEF2E2554F554E4F5BB
:1029AC0052E54E540EFFC313901EDE93FFC454F039
:1029BC004252E54E5401FF33333354F84252E55240
:1029CC005408FFC313901ECE93FFE55254C0FEC4AF
:1029DC00540F932F042553F553E55254A0FEC454C1
:1029EC000F932F042554F554E5535401FF25E0258E
:1029FC00E04252E5545401FF25E04252E552540E98
:102A0C00FFC313901EDE934252AB4F0551E551AA02
:0D2A1C00507002055014F9E552121A2022E4
:102A290030014FE56D704B74A7257BF582E434685E
:102A3900F583E0FD7B017A6A79A1AF741228CC7520
:102A490074FF857D6D057BD57602C201906693E0A2
:102A5900FCA3E0FDA3E0FEA3E0FFE4FAF9F8EF240C
:102A690001FFEA3EFEE93DFDE83CFC906693121B3E
:102A79005422200503300F493005117B017A6A7908
:102A8900A17DFF7FFB1228CCC205800F7B017A6AEA
:102A990079A17DFE7FFB1228CCC20F906693E0FCE2
:102AA900A3E0FDA3E0FEA3E0FFE4FAF9F8EF2401B7
:102AB900FFEA3EFEE93DFDE83CFC906693121B549B
:102AC900229066A2E0FF04F0EF75F002A424A8F9B1
:102AD900746A35F0FA9068A47401F0A3EAF0A3E9E6
:102AE900F09068A4E0FBA3E0FAA3E0F91219DA2058
:102AF900E6099066A2E0C394FB40C69066A2E0FF97
:102B0900B4FB17E4F0E56D6002156D906AA174EEEF
:102B1900F0A37447F0A37414F022EF14FF9000019E
:102B29001219F3FD7B017A6A79A11228CC9068A465
:102B3900E0FBA3E0FAA3E0F91219DA54BF121A2054
:102B4900E56D6002156D906693E0FCA3E0FDA3E0DE
:102B5900FEA3E0FFE4FAF9F8EF2401FFEA3EFEE9FB
:0E2B69003DFDE83CFC906693121B54D2902276
:1016840030072DC3E5279547FFE5269546FED3EFA2
:101694009440EE940040197B087D40AF47AE46125B
:1016A400317DE5472440FFE43546540FF5468F4726
:1016B400201405D291D29022200303021927E54376
:1016C4005438653A602C9067A9E064036024E53AD5
:1016D40024085438F53A131313541F242AF8E6FF48
:1016E400E0FE04F074A42EF582E4346AF583EFF08E
:1016F40080CC9067A9E064036003021946F0906A05
:10170400A4E064EE701EA3E0B44719A3E0B414147B
:10171400201E030219097E1E7F4DE4FBFDFC122CE2
:10172400B3021909301E0D7E1E7F567C6A7DA47B90
:1017340003122CB3E49066A3F090669FF0906AA421
:10174400E0FF54E0FE9066A3F0EF540EFF25E04E58
:10175400FFF0906AA5E0FE54C0FDC4131354034F78
:10176400FF9066A3F0EE5420FE25E025E0FE90668F
:101774009FF0906AA5E0540EFD33333354F84EFEC7
:1017840090669FF0906AA6E0FD54E0FCC4540F4EAE
:10179400FE90669FF0ED5408FD131313541F4EFE84
:1017A400F0FD7B017A6679A61228CC9066A6E0FF4C
:1017B400906AA4E0B507189066A7E0FF906AA5E0D8
:1017C400B5070C9066A8E0FF906AA6E06F60382029
:1017D4001C0D7E1E7F607C6A7DA47B03122CB3905B
:1017E4006697E0FCA3E0FDA3E0FEA3E0FFE4FAF9C2
:1017F400F8EF2401FFEA3EFEE93DFDE83CFC90667B
:1018040097121B5402190990668FE0FCA3E0FDA314
:10181400E0FEA3E0FFE4FAF9F8EF2401FFEA3EFE5C
:10182400E93DFDE83CFC90668F121B549066A3E0F2
:10183400FF2402605114606C8000EFC394F94003EC
:10184400021909AE79057974A12EF582E43469F59B
:1018540083EFF090669FE0FFAE79057974A12EF5D1
:1018640082E43469F583EFF0301C030219097E1E0B
:101874007F6C749F2579F582E43469AD82FC7B0228
:10188400122CB302190990669FE0FF6017300B0217
:10189400D20FD20B9066A4EFF0E49066A0F0906CA7
:1018A400A8F08061300B5E9066A4E0604290669F71
:1018B400E0FF906CA8E0FE04F074AA2EF582E434F4
:1018C40067F583EFF09066A0E02FF09066A4E01433
:1018D400F0201C317E1E7F767C667D9F7B02122C5D
:1018E400B390669FE0FF7E007D0212309C8016C29A
:1018F4000B90669FE0FFA3E0B50708D20ED205D295
:10190400108002D20F0570E570641F7035C203C2E7
:1019140091F540F53FF53EF53DD22AE5796023D2B5
:101924000E801F202A1CC20EE49067A9F0D203F592
:1019340079F570D291201C0A7E1E7F80FBFDFC127B
:101944002CB3300C6CE54424085438FFE53B543880
:101954006F60047E0180027E00E57A640360047D8A
:101964000180027D00EE5D601F74A1257AF582E49A
:10197400346AF583E0FEE544131313541F2432F84C
:10198400A6068F44057A80BDE57A64037047057323
:10199400E573B42007C20CC290D20822E4F57A128F
:1019A4002A29201C307E1E7F91E4FBFDFC122CB3FF
:1019B40022E4F57A906AA17466F0A37496F0A37495
:1019C40099F0201C0B7E1E7F9CE4FBFDFC122CB3C3
:0619D400D20CE4F57322C1
:0B3F6100300D05C20D7F01227F002201
:033F6C00C2AE22C0
:1035F100020879E493A3F8E493A34003F68001F26F
:1036010008DFF48029E493A3F85407240CC8C333DA
:10361100C4540F4420C8834004F456800146F6DFA9
:10362100E4800B0102040810204080903F10E47EEA
:10363100019360BCA3FF543F30E509541FFEE4939E
:10364100A360010ECF54C025E060A840B8E493A365
:10365100FAE493A3F8E493A3C8C582C8CAC583CA90
:10366100F0A3C8C582C8CAC583CADFE9DEE780BE48
:013F2B000095
:1019DA00BB010689828A83E0225002E722BBFE020B
:0919EA00E32289828A83E493223E
:1019F300BB010CE58229F582E5833AF583E02250A9
:101A030006E92582F8E622BBFE06E92582F8E222F2
:0D1A1300E58229F582E5833AF583E493220C
:101A2000BB010689828A83F0225002F722BBFE01A5
:021A3000F3229F
:101A3200F8BB010DE58229F582E5833AF583E8F0EA
:101A4200225006E92582C8F622BBFE05E92582C896
:021A5200F2227E
:101A540075F008758200EF2FFFEE33FECD33CDCC49
:101A640033CCC58233C5829BED9AEC99E5829840CC
:101A74000CF582EE9BFEED9AFDEC99FC0FD5F0D6A9
:101A8400E4CEFBE4CDFAE4CCF9A88222B800C1B9D3
:101A94000059BA002DEC8BF084CFCECDFCE5F0CB11
:101AA400F97818EF2FFFEE33FEED33FDEC33FCEB4A
:101AB40033FB10D703994004EB99FB0FD8E5E4F905
:101AC400FA227818EF2FFFEE33FEED33FDEC33FCF2
:101AD400C933C910D7059BE99A4007EC9BFCE99AE6
:101AE400F90FD8E0E4C9FAE4CCFB2275F010EF2F2B
:101AF400FFEE33FEED33FDCC33CCC833C810D7072B
:101B04009BEC9AE899400AED9BFDEC9AFCE899F865
:0E1B14000FD5F0DAE4CDFBE4CCFAE4C8F922F8
:0E1B2200C3E49FFFE49EFEE49DFDE49CFC22D4
:101B3000EB9FF5F0EA9E42F0E99D42F0E89C45F00B
:011B40002282
:101B4100E8600FECC313FCED13FDEE13FEEF13FF82
:031B5100D8F122A6
:0C1B5400ECF0A3EDF0A3EEF0A3EFF02204
:101B6000A8828583F0D083D082121B77121B771254
:101B70001B77121B77E473E493A3C583C5F0C58379
:101B8000C8C582C8F0A3C583C5F0C583C8C582C8CF
:011B90002232
:10132800E5622456F8E6056222785330280278569A
:10133800E475F001121BE00219DA2021EB7F2ED2AE
:10134800218018EF540F2490D43440D4FF30250B5B
:10135800EF24BFB41A0050032461FFE5636002154F
:10136800630566E5667002056530280D7853E475F7
:10137800F001121BE0EF021A20023D557403D22837
:101388008003E4C228F5628B538A548955E4F563D7
:10139800F565F566E56360077F2012136380F575D0
:1013A80064FFC222C221C223C224C226C227C22984
:1013B800121331FF700D3028057F00121374AF66C9
:1013C800AE6522B4255FC2D5C225121331FF24D0E1
:1013D800B40A00501A75F00A786330D50508B6FFCC
:1013E8000106C6A426F620D5047002D22480D9248A
:1013F800CFB41A00EF5004C2E5D225021574D222E8
:1014080080C6D22180C0D22380BCD2D580BAD22651
:1014180080B47F201213632023077401B563004052
:10142800F1121328FF12136302139CD229D22780CA
:1014380095121328FB121328FA121328F94A4B7035
:101448000679457A167BFF20232EE563602A7E0005
:101458008E827583001219F360060EEE656470F0D3
:10146800C2D5EBC0E0EAC0E0E9C0E0EE1215BBD09F
:10147800E0F9D0E0FAD0E0FB1219DAFF60AAEBC07D
:10148800E0EAC0E0E9C0E0121363D0E02401F9D03B
:10149800E03400FAD0E0FBE5640460DCD564D98070
:1014A800877BFF7A1579B7D223809C7910800279DF
:1014B80008C227C2298008D2D5790A8004790AC2CD
:1014C800D5E564047002F564E4FAFDFEFF12132802
:1014D800FC7B08202213121328FD7B1030210A12EE
:1014E8001328FE121328FF7B20EC3382D592D550A7
:1014F80013C3E43021069FFFE49EFEE42022039DEF
:10150800FDE49CFCE4CBF8C222EC700CCFCECDCC31
:10151800E824F8F870F38017C3EF33FFEE33FEEDDD
:1015280033FDEC33FCEB33FB994002FB0FD8E9EBBE
:10153800302205F8D0E0C448B222C0E00AEC4D4E93
:101548004F78207B0070C2EAB5640040BCC0E0124E
:1015580015BDD0F0D0E0202204C4C0E0C4B222C03F
:10156800F012134CD0F0D5F0EB02139C121C3F1470
:10157800395314B358140A4C14064214B74F14BF05
:0F1588004414BF49141F4314C55514A94614A990
:101597004514A947166550140E2D14122E14352B19
:1015A700141623143320164E2A13CE480000142D88
:1015B7003F3F3F00790AA2D5202414302609B910ED
:1015C700020404B9080104A2D5202702500104200F
:1015D70023689223B563005034C0E07F203024197C
:1015E7007F30A22372277226500F121614C223C20D
:1015F70027C226C2297F30800F302603E9C0E012B8
:101607001363302603D0E0F9D0E0B563CC3026175A
:101617007F30B9100C1213637F583025077F78800D
:1016270003B908031213633023057F2D0213637F69
:10163700202029F87F2B2027F322922380CF286EA2
:10164700756C6C2900D2221213283022F8C2227836
:101657006330D50108F60213CE2D504349581213B3
:10166700282403B405004001E49016609312135434
:0D167700743A121354D2247563040214B3A4
:1022A1008B578A588959E4F563F562F561F560F554
:1022B1005EF55FE55B455C455A6012EBC0E0EAC044
:1022C100E0E9C0E0AB5AAA5BA95C121BF0AB570571
:1022D10059E559AA587002055814F91219DAF5642A
:1022E100C394094007E564D3940D40E1E56464209B
:1022F10060DBE564B42D05435F038016E564B42B10
:1023010005435F01800C74FF2559F55974FF355859
:10231100F558E55D60046410703FAB57AA58A959A0
:102321001219DA64306009E55D702E755D0A802945
:102331009000011219F3FF64786004EFB45813435D
:102341005F01755D1074022559F559E43558F5584A
:102351008007E55D7003755D08AB570559E559AA1E
:10236100587002055814F91219DAF564C3946140E2
:102371000AE564D3947A50035364DF74D02564F57D
:1023810064C3940A400CE5649411406D74F92564AA
:10239100F564E564D3955D5060435F0185636885AD
:1023A1006267856166856065AF5D7E00E4FCFDABBB
:1023B10063AA62A961A860121B91C8ECC8C9EDC9E2
:1023C100CAEECACBEFCBE4FCFDFEEB2564F563EE70
:1023D1003AF562ED39F561EC38F560AF63AE62ADA7
:1023E10061FCAB68AA67A966A865D3121B305003CC
:1023F10002235A435F0402235AE55F20E003E4808D
:102401002DE55B455C455A601EAB57E55924FFF944
:10241100E55834FFFAEBC0E0EAC0E0E9C0E0AB5AAE
:10242100AA5BA95C121BF0E55F30E20774FFFFFEB7
:10243100FDFC22E55FAF63AE62AD61AC6030E103EC
:04244100021B222236
:101B9100E88FF0A4CC8BF0A42CFCE98EF0A42CFCF3
:101BA1008AF0EDA42CFCEA8EF0A4CDA8F08BF0A471
:101BB1002DCC3825F0FDE98FF0A42CCD35F0FCEBD0
:101BC1008EF0A4FEA9F0EB8FF0A4CFC5F02ECD3995
:0F1BD100FEE43CFCEAA42DCE35F0FDE43CFC2202
:101BE000FAE6FB0808E6F925F0F618E6CA3AF62206
:101BF000BB011A89828A83D0F0D0E0F8D0E0F9D016
:101C0000E0FAD0E0FBE8C0E0C0F0021C6E5016E93C
:101C1000F8D083D082D0E0F9D0E0FAD0E0FBC082E7
:101C2000C083021C65BBFE16E9F8D083D082D0E0E9
:0F1C3000F9D0E0FAD0E0FBC082C083021C77221B
:101C3F00D083D082F8E4937012740193700DA3A334
:101C4F0093F8740193F5828883E473740293686048
:061C5F00EFA3A3A380DF48
:091C6500EBF608EAF608E9F622A4
:091C6E00EBF0A3EAF0A3E9F02277
:091C7700EBF208EAF208E9F2229E
:00000001FF
